:10000000370101007128A948730000008280148123
:10001000988133E6E60009C685050505E389E6FE15
:1000200013351600828052B82A846D2C2A945D2CD8
:10003000E36F85FE52BE8AB8612C25C113044006C9
:1000400093045006130940079309300619A0492468
:1000500029C501455D240808C1450A86C146B52C5D
:1000600003450101E31585FE03451101E31195FEEA
:1000700003452101E31D25FD03453101E31995FCED
:1000800003454101E31535FD03455101E31125FD0C
:10009000034561014DFD05458ABE0545B92C8ABC65
:1000A000FAB81305C033012C130520352924130495
:1000B00040379305A037228539241305E03793058F
:1000C00030381124130570389305C038ED2A130B0E
:1000D000F038930B60397EAFFD22192C130D4006CA
:1000E000930D50069304400713093006930A2043EA
:1000F000130CE043930910441305A0396D2A0545FC
:10010000ED2A1305003A452AE12221C50145F522D1
:100110000808C1450A86C146C92203450101E31505
:10012000A5FF03451101E311B5FF03452101E31DBF
:1001300095FC03453101E319B5FD03454101E31584
:1001400025FD03455101E31195FC034561014DFD7A
:1001500021A005455D224DBF1305103BA92A01458D
:10016000692A22859305203DB92A1305903DA122D5
:10017000952A130A2500BD22E36F45FF1305E037DA
:100180009305803E89221305B03E3522A12A130A29
:100190002500892AE36F45FF7EAC35221305503FC9
:1001A000192A8922130A3500352AE36F45FF130502
:1001B000703893051040012A13056040ED281D2278
:1001C000130A45000522E36F45FF1305E037930549
:1001D0003038D52813052041F9285A859305D04198
:1001E000DD2013053042C12821223D4A09A80545DA
:1001F0002922014519227D1A1375FA0F3DC9937CF6
:10020000FA0F56854D2866855D2062856D20D928B8
:10021000930C1500C128E36F95FF5D2869D901454E
:10022000E9280808C1450A86C14645280345010159
:10023000E315A5FF03451101E311B5FF03452101B6
:10024000E31D95FC03453101E319B5FD034541016B
:10025000E31525FD03455101E31195FC03456101BB
:100260004DFD612871204E85B920614A1375FA0F42
:1002700059F51305604581207EAFB1201305104666
:100280001D28130570389305C03835281305E0463E
:100290001D208928130A2500B120E36F45FF228520
:1002A0009305A0370D20130580473120B1B585484F
:1002B0007300000082809148730000008280AD4886
:1002C0007300000082809308100873000000828091
:1002D0009308500873000000828093087008730030
:1002E00000008280732510C08280732500C0828048
:1002F000930860087300000082800589F322008063
:1003000093920248B3E2A2007390028082809548E3
:100310007300000082809308000873000000828050
:10032000A148730000008280930830087300000029
:100330008280930840087300000082804445205268
:1003400061696C726F61642043726F7373696E6769
:100350000A00666F72205256436F6E74726F6C6C37
:1003600065720A496E697469616C697A696E6720A1
:1003700048570A006C69676874004F46460062651A
:100380006C6C006F66660067617465007570007361
:1003900069676E616C005245440049646C650A00EF
:1003A0004C696768747765696768743A204F6E0AAC
:1003B00000547261696E2064657465637465640AD3
:1003C0004C696768747765696768743A204F666638
:1003D0000A0059454C4C4F57004C696768743A20E5
:1003E00059656C6C6F770A006F6E0042656C6C3AF1
:1003F000204F6E0A004C696768743A205265640A9F
:1004000000646F776E00476174653A20446F776EC1
:100410000A0042656C6C3A204F66660A00475245F6
:10042000454E005369676E616C3A20477265656E90
:100430000A0054696D656F757420696E2000730A37
:100440000054696D6520726573657420627920744B
:100450007261696E0A0054696D6564206F75740A73
:10046000005369676E616C3A205265640A00476107
:1004700074653A2055700A004C696768743A204FD9
:0404800066660A00A2
:00000001FF
